:020000040000FA
:02000000E329F2
:080008008F00030E8E00AF0310
:1000100003190B2836281330AF003C205920A220AA
:100020001B1C18289303031D18286430930094099F
:1000300002219003FF301002031D36280930900082
:100040009103FF301102031D3628093091009203FD
:10005000FF301202031D362803309000013091005A
:10006000053092001C18D1201D18CE200B110E0E49
:1000700083008F0E0F0E09001D18080017180800C6
:100080001918080015184E28061808001E101B1411
:100090001C101D10FA309600151408009603031D5D
:1000A000080015108D0A05300D02031D08008D0192
:1000B00008001D180800151808001918080017185E
:1000C0006B28861808001E101B141C101D1096307B
:1000D0009800171408009803031D0800171000303B
:1000E0000D02031D7A289F0A0A301F02031D080013
:1000F0009F01080001300D02031D8528A00A06306B
:100100002002031D0800A001080002300D02031D9B
:100110009028A10A0A302102031D0800A10108004D
:1001200003300D02031D9B28A20A06302202031D84
:100130000800A2010800A30A0A302302031D0800D8
:10014000A301080017180800151808001918C92875
:10015000861B08001B1CBE28FA309A0019141E10BA
:100160001B101C141D101F08A4002008A500210846
:10017000A6002208A7002308A80008001D1C0800EC
:10018000FA309A0019141E141B101C101D100613AF
:1001900008009A03031D0800191008004030860665
:1001A0000800A803FF302802031DF7280930A80023
:1001B000A703FF302702031DF7280530A700A60379
:1001C000FF302602031DF7280930A600A503FF30E3
:1001D0002502031DF7280530A500A403FF302402E3
:1001E000031DF7281E101B101C101D1408002408E6
:1001F0009F002508A0002608A1002708A2002808C3
:10020000A30008001D1C052907291E1C0D29A90192
:10021000AA01AB01AC01AD014C291B1C3F29141CE8
:10022000342900300D02031D18290F30A9004C2974
:1002300001300D02031D1F290F30AA004C29023086
:100240000D02031D26290F30AB004C2903300D028F
:10025000031D2D290F30AC004C2904300D02031D65
:100260004C290F30AD004C291F08A9002008AA0016
:100270002108AB002208AC002308AD004C291C1C4F
:100280004C292408A9002508AA002608AB00270845
:10029000AC002808AD004C298C03FF300C02031D74
:1002A000532904308C0000300C02031D5C291E30E1
:1002B00085002908AE00802901300C02031D652944
:1002C0001D3085002A08AE00802902300C02031D73
:1002D0006E291B3085002B08AE00802903300C02EC
:1002E000031D7729173085002C08AE0080290430C3
:1002F0000C02031D80290F3085002D08AE008029D7
:1003000000302E02031D892906118611061286125D
:10031000080001302E02031D9229061586110612CF
:100320008612080002302E02031D9B290611861535
:1003300006128612080003302E02031DA42906159A
:10034000861506128612080004302E02031DAD2900
:100350000611861106168612080005302E02031DAE
:10036000B6290615861106168612080006302E02DA
:10037000031DBF29061186150616861208000730D0
:100380002E02031DC82906158615061686120800BA
:1003900008302E02031DD129061186110612861679
:1003A000080009302E02031DDA29061586110612EF
:1003B000861608000F302E02031D0800061586154C
:1003C0000616861608008312850186018316003002
:1003D0008100003085008330860083120C30840059
:1003E0008001840A50300402031DF029033090007C
:1003F00001309100053092001330AF0004308D00C1
:10040000FA30960096309800FA309A0064309300E3
:0E04100006131E148101A0308B000E2A0E2A46
:02400E00F23F7F
:104200002800430029004600610062007200690036
:10421000630065002000530069006E0063006500C4
:10422000720065002000300032002F0030003300A3
:0A4230002F0032003000300037008C
:00000001FF
